:100000000C9499030C94B6030C94B6030C94B603A9
:100010000C94B6030C94B6030C94B6030C94B6037C
:100020000C94B6030C94B6030C94B6030C94B6036C
:100030000C94B6030C94B6030C94B6030C940F0BFB
:100040000C94B6030C94B6030C94AC170C94B60342
:100050000C94B6030C94B6030C94B6030C94B6033C
:100060000C94B6030C94B6030C94B6030C94B6032C
:100070000C94B6030C94B6030C94C4150C94B603FC
:100080000C9403140C94B6030C94B6034F4B0A0063
:100090004552524F520A00494E56414C49440A00BB
:1000A00008200800524F42494E3E200042444D492C
:1000B00043524F203A204D41565249432D4949421F
:1000C000203A20524F42494E2054657374204361B8
:1000D00073652056657273696F6E2032000A0A528A
:1000E0004F426F7420496E646570656E64656E740E
:1000F000204E6574776F726B2028524F42494E290B
:100100000A0A000A76616C696420636F6D6D616E26
:1001100064733A0A0A2020706B745B3C666C6167FA
:10012000733E5D203C69643E205B3C646174613ECB
:100130005D0A0A2020202053656E642061207061D2
:10014000636B657420746F206E6F6465203C696416
:100150003E2C20616C6C206461746120666F6C6C55
:10016000696E67207468652069732073656E7420FA
:100170006173207468650A202020207061636B65BC
:100180007420646174612E2020466C616773206363
:10019000616E20626520276327203D20636F6C6CB1
:1001A0006973696F6E206465746563742C202761C0
:1001B00027203D20726571756573742061636B2C17
:1001C0000A202020206F7220276927202D207265A9
:1001D00071756573742069642E20204578616D7097
:1001E0006C65733A0A0A202020202020706B74204E
:1001F000422074657374207061636B6574202D20D8
:1002000073656E64206E6F726D616C207061636BDC
:10021000657420746F206E6F646520420A0A202086
:1002200020202020706B74692042202D207265717F
:100230007565737420616E20494420726573706F18
:100240006E73652066726F6D206E6F646520420A62
:100250000A202020202020706B7463692042202D0A
:10026000207265717565737420616E204944207237
:100270006573706F6E73652066726F6D206E6F644C
:100280006520422C2075736520636F6C6C697369FF
:100290006F6E20646574656374696F6E0A0A20204E
:1002A00020202020706B74632042207465737420BA
:1002B0007061636B6574202D2073656E64206E6FB2
:1002C000726D616C207061636B657420746F206E59
:1002D0006F646520422C2075736520636F6C6C69B8
:1002E00073696F6E20646574656374696F6E0A0A62
:1002F000202020202020706B7461204220746573C0
:1003000074207061636B6574202D2073656E6420AA
:100310006E6F726D616C207061636B657420746FB9
:10032000206E6F646520422C207265717565737450
:100330002041434B20726573706F6E73650A0A200B
:10034000206964205B3C69643E5D0A0A202020200D
:10035000536574207468652063757272656E7420CD
:100360006E6F6465277320696420746F203C696434
:100370003E2E20204966203C69643E206973206F30
:100380006D69747465642C20746865206E6F646593
:10039000732063757272656E740A20202020696470
:1003A00020697320646973706C617965642E202004
:1003B0004578616D706C653A0A0A20202020202063
:1003C00069642041202020202D20736574207468EA
:1003D00065206E6F646520696420746F2027412753
:1003E00020286865782030783431290A0A20206373
:1003F0006F6C6C696465203C6E6F6465313E203CB7
:100400006E6F6465323E202D20617474656D70746A
:1004100020746F206361757365206120636F6C6C5D
:100420006973696F6E206F6E20746865206E6574E5
:10043000776F726B0A0A202020204669727374203D
:1004400073656E6420616E20494420726571756524
:10045000737420746F203C6E6F6465313E20746F3E
:1004600020656C69636974206120726573706F6EBA
:10047000736520616E640A20202020656E7375729A
:100480006520746861742061207061636B657420FD
:1004900077696C6C20736F6F6E2062652070726577
:1004A00073656E74206F6E20746865206275732E9C
:1004B00020205468656E2C0A20202020696D6D650F
:1004C00064696174656C7920626567696E20696E24
:1004D0006469736372696D696E6174656C792062B9
:1004E0006C617374696E67207061636B65747320EF
:1004F000746F203C6E6F6465323E20746F0A20205A
:10050000202074727920616E642067656E65726167
:100510007465206120636F6C6C6973696F6E2077FE
:100520006974682074686520494420726577706F2B
:100530006E73652066726F6D203C6E6F6465313E30
:100540002E0A0A20202020546865206E6F646520E2
:100550003C6E6F6465313E206E6565647320746F18
:10056000206265206F6E207468652062757320615B
:100570006E64206F7065726174696F6E616C2C209F
:100580006275740A202020203C6E6F6465323E2024
:100590006E656564206E6F7420626520707265738D
:1005A000656E7420666F7220746869732074657359
:1005B000742E0A0A20207363616E202D20736361FC
:1005C0006E2074686520627573206C6F6F6B696E46
:1005D0006720666F72206E6F646573206279206990
:1005E000737375696E6720616E204944207265716E
:1005F0007565737420666F720A20202020202020E9
:10060000202065616368206164647265737320658E
:100610007863657074206F7572206F776E20616EDD
:1006200064206C6F6F6B696E6720666F72207265F5
:1006300073706F6E7365732E0A0A202070696E677F
:10064000203C6E6F64653E202D2073656E64203102
:100650003030207061636B65747320746F20746830
:100660006520737065636966696564206E6F646593
:100670002C20656C69636974696E6720610A2020AB
:1006800020202020202020726573706F6E736520FB
:100690006261636B3B2063616C63756C61746520A0
:1006A00074686520746F74616C2074696D65207462
:1006B000616B656E20616E64207265706F7274206C
:1006C000616E790A2020202020202020206572726F
:1006D0006F72730A0A202076202D20746F67676C72
:1006E0006520766572626F7365206D6F64653B206F
:1006F0007768656E20656E61626C65642C20696E3A
:10070000636F6D696E67207061636B6574732061E0
:100710007265206563686F65640A202020202020B0
:10072000746F20746865207465726D696E616C0AFF
:100730000A0011241FBECFEFD0E1DEBFCDBF15E010
:10074000A0E0B1E0EAE1F2E400E00BBF02C00790F4
:100750000D92A430B107D9F717E0A4E0B5E001C0CD
:100760001D92A839B107E1F70C9493120C94000084
:100770002F923F924F925F926F927F928F929F92B1
:10078000AF92BF92CF92DF92EF92FF920F931F939F
:10079000CF93DF93CDB7DEB726970FB6F894DEBFC1
:1007A0000FBECDBF5C016A017B01522E180127FFED
:1007B00002C0552405C085E2821714F485E2582E44
:1007C000D5019896BE83AD8320E030E040E050E054
:1007D000C701B6010E94E61E882354F4F10180810E
:1007E0009181826091838083F7FAF094F7F8F09416
:1007F000AE014F5F5F4FC701B6010E94461F3B012C
:100800004C01E980FA800B811C8120E030E040E05F
:1008100050E0C801B7010E94E61E8823E9F1CD80AF
:10082000DE80442428C02DEC3CEC4CEC5DE3C80198
:10083000B7010E94761FAE014F5F5F4F0E94461FB7
:100840002AE939E941E251E40E94761F0E94CB1E59
:10085000605DD6016E936D014394E980FA800B814F
:100860001C8120E030E040E050E0C801B7010E9468
:10087000E61E882319F0AC14BD04A8F2750106C069
:10088000F60181916F01D7018D937D01ED81FE818C
:10089000CE16DF06A8F329C020E030E040E050E0AB
:1008A000C401B3010E94E91E18161CF0750144240E
:1008B0001CC0442403C04A943701480120E030E0C2
:1008C00040E251E4C401B3010E94761F7B018C0118
:1008D00020E030E040E85FE30E94E61E87FDEBCFBA
:1008E000E982FA820B831C837501D1014D915C91E1
:1008F00053FF13C0BDEF4B1684F0242D332727FD83
:100900003095852D992787FD9095019628173907F1
:1009100024F45460F10151834083D1018D919C9165
:1009200092FD08C05394052D112707FD10950A0D5F
:100930001B1D0CC0052D112707FD10950A0D1B1D51
:10094000842D992787FD9095080F191F0A151B05FF
:10095000D8F4F5014CC020E030E040E251E4C4019D
:10096000B3010E94761FAE014F5F5F4F0E94461F8A
:100970003B014C0169817A818B819C810E94CB1E55
:10098000605DD7016D937D010E151F0528F0ED8187
:10099000FE81EE16FF06F8F28D819E810817190779
:1009A00018F0F50117A224C0D8018C918B5F8C93AD
:1009B000F80131E318C020E3D8012C93A016B1064A
:1009C00028F48E918D018F5F8C930DC0D8013C93DC
:1009D0004394D1018D919C9192FF05C0AE16BF0644
:1009E00008F420833196D8018C918A3324F7108241
:1009F000842D992787FD909526960FB6F894DEBF33
:100A00000FBECDBFDF91CF911F910F91FF90EF905F
:100A1000DF90CF90BF90AF909F908F907F906F901E
:100A20005F904F903F902F9008952F923F924F925A
:100A30005F926F927F928F929F92AF92BF92CF926E
:100A4000DF92EF92FF920F931F93CF93DF93CDB777
:100A5000DEB7EE970FB6F894DEBF0FBECDBFCC2445
:100A6000DD2476013C017EAF6DAF5A011A821982F6
:100A7000FC0117821682838181FDF3C38FEF9FEF04
:100A800016C409811A8100FFD3C3842D80538A3094
:100A9000D0F4F0E34F1631F4552021F403FD02C0E9
:100AA000116075C18AE0252D2802C0011124542C43
:100AB000580E30ED530E57FE02C04FE7542E03FD83
:100AC000CAC3352CC8C3442D45564CAF433028F01B
:100AD000842D8554833008F0FCC0C501049698AF7E
:100AE0008FABF501C080D180E280F38003FD02C0AE
:100AF00036E0532E077B1A83098346015701A7016D
:100B00009601C701B6010E94B8188823C1F08EE48F
:100B10008D838B8381E48C839E012A5F3F4F3AAFA4
:100B200029AF3CAD333008F07AC28B81805E8B8375
:100B30008C81805E8C838D81805E8D8370C2C701C5
:100B4000B6010E943D1F892BE9F089E48D838EE474
:100B50008C8386E48B8320E030E040E050E0C701E6
:100B6000B6010E94E61E87FD06C0AE014A5F5F4FD8
:100B70005AAF49AFD6CF8DE28E83CE0107969AAF9A
:100B800089AFCFCFC80192609A838983E7E44E167C
:100B900009F449C0E41544F0F5E44F1679F026E471
:100BA000421609F042C31DC036E64316D1F047E6AF
:100BB0004416C9F155E6451609F037C38E010F5F9B
:100BC0001F4F252DB501A401CE010F960E94B80339
:100BD000282E8CEF380E15140CF43A94DE011F9673
:100BE00015C094609A8389838E010F5F1F4F252D56
:100BF000B501A401CE010F960E94B803282E15144A
:100C00000CF43A94DE011F96121444F4FD01019095
:100C10000020E9F73197CE2ECA1A02C0C52CC39422
:100C2000BAAFA9AF7DC1552011F0252D01C021E03B
:100C300098609A8389838E010F5F1F4FB501A401CD
:100C4000CE010F960E94B803282E89819A8192FFC7
:100C50001EC0822D850D8150282FA82FBB27A7FDF0
:100C6000B095AC0FBD1F1F9605C08C9111972150F8
:100C7000803331F4622F27FD23C02215B4F703C35C
:100C8000C62E562E5218539400C3C92E17C0252DB8
:100C9000E52DFF27E7FDF095EC0FFD1F3F9606C001
:100CA00080813197292F2150803379F7922F1216A6
:100CB000BCF3522EC22E222309F4EFC2592EEDC2EC
:100CC000E22FFF27E7FDF095EC0FFD1F108A55245A
:100CD00099CFC8018870907003FF04C0552011F4AB
:100CE00021E0522EE9E64E1609F493C0E4153CF1DA
:100CF000F3E54F1609F474C0F415ACF02BE242167C
:100D0000E1F1241544F030E24316D1F143E24416F8
:100D100009F080C23FC05DE24516C1F18EE248167F
:100D200009F078C239C093E64916E1F1E4E64E16BF
:100D300009F46FC0F8E54F1609F06CC29FC020E7B8
:100D4000421609F496C0241544F03CE6431641F1DE
:100D50004FE6441609F05EC20DC055E7451609F48A
:100D60008FC0E8E74E1609F489C0F3E74F1609F083
:100D700051C221C028E02BAF83C000611A830983D0
:100D800089819A8180629A83898365C200681A8307
:100D9000098361C20064FBCF08601A83098352C2D1
:100DA0000460F5CFA5014E5F5F4F58AF4FABF50123
:100DB000C0803A9434C1F501C080D180892B41F0C4
:100DC000652D772767FD7095C6010E949E1C18C08F
:100DD000F60101900020E9F73197EC19EBAF11C053
:100DE000F501C080D180892B41F0652D772767FD03
:100DF0007095C6010E944A1C03C0C6010E94411C96
:100E00008BAF95012E5F3F4F38AF2FAB3BAD331A01
:100E100006C102FF0BC0A5014C5F5F4F58AF4FAB3F
:100E2000F50160817181828193810EC095012E5FF1
:100E30003F4F38AF2FABF501808191819C01B90103
:100E4000882777FD8095982F6B017C0197FF0BC059
:100E500002601A830983F094E094D094C094C11C7A
:100E6000D11CE11CF11C89819A818F7B9A83898333
:100E700027C000641A83098398E7492E30E13BAF0D
:100E800029813A8122FF0BC0A5014C5F5F4F58AF0B
:100E90004FABF50160817181828193810CC0A50106
:100EA0004E5F5F4F58AF4FABF50180819181AC0130
:100EB000BA01882799276B017C012F7C3A8329830B
:100EC00087017601CE0103969AAF89AF9BADA92E1B
:100ED000BB24CC24DD24C801B701A60195010E94E2
:100EE00054206A301CF0640D615201C0605DE9ADB0
:100EF000FAAD6193FAAFE9AFC801B701A601950158
:100F00000E94542079018A012115310541055105BE
:100F100011F7CC24DD247601CE010396C9ACC81AA2
:100F200049815A81CA0182739070892B09F03A94E1
:100F300046FF07C0FBADF03111F482E001C081E053
:100F4000381A43FF10C0252D332727FD30958C2DEF
:100F500099278217930724F0477F5A83498303C058
:100F60005C18351801C03C1840785170452B69F465
:100F7000832D06C0B30180E290E00E94F91C812F0E
:100F8000182F11501816B4F3312E89819A8181FFE0
:100F900004C0B3018DE290E00BC084FF04C0B30134
:100FA0008BE290E005C085FF05C0B30180E290E0D0
:100FB0000E94F91C89819A8186FF0FC0B30180E3EA
:100FC00090E00E94F91C2BAD203139F4B301842D3F
:100FD000992787FD90950E94F91C89819A8190FF3D
:100FE0000DC0832D06C0B30180E390E00E94F91C80
:100FF000812F182F11501816B4F3312E89819A8140
:1010000083FF0DC0252D06C0B30180E390E00E9450
:10101000F91C212F122F11501216B4F3512E898171
:1010200087FD0DC0832D06C0B30180E290E00E94D1
:10103000F91C812F182F11501816B4F3312E33E6F6
:10104000431631F4B3018C2D992787FD9095BEC0CE
:1010500043E74416B1F4460156011BAD09C0F50142
:1010600081915F01B301992787FD90950E94F91C3A
:101070001150A8F76401FBADCF0ED11C2FEF2BAFA1
:10108000B8C033E54316B1F446018601BBAC08C0D5
:10109000F8018491B30199270E94F91C0F5F1F4F3B
:1010A000BA94FFEFBF16A1F764012BADC20ED11C9D
:1010B000FBAF9FC089819A8191FD03C009AD1AAD34
:1010C00091C092FF1DC01214BCF4A9ACBAAC122D91
:1010D00009C0F50181915F01B301992787FD9095C2
:1010E0000E94F91C1150A8F729AD3AAD220D311D0F
:1010F0003AAF29AF22240FC0B30180E390E009C0CA
:10110000E9ADFAAD8191FAAFE9AFB301992787FD57
:1011100090950E94F91C15142CF4B3018EE290E016
:101120000E94F91C89819A8192FD06C017C0B30103
:1011300080E390E00E94F91C2394822D815087FF68
:101140000DC05A94852D8F5F18168CF307C0B3011C
:10115000892F992787FD90950E94F91CE9ADFAAD7A
:101160009191FAAFE9AF992329F05A94852D8F5FB9
:1011700018166CF389819A8192FD3BC0B301842DCE
:10118000992787FD90950E94F91C2A9427FE07C095
:10119000B3018DE290E00E94F91C219405C0B301D7
:1011A0008BE290E00E94F91C6AE070E0822D9927A2
:1011B00087FD90950E9441206B017C01CB01C09678
:1011C000B3010E94F91CB301C701C0960E94F91C2B
:1011D00010C0F80182918F01B301992787FD909586
:1011E0000E94F91CCE0103960817190791F71AAF50
:1011F00009AF898187FF17C0832D06C0B30180E244
:1012000090E00E94F91C812F182F11501816B4F38A
:10121000312E09C0B301842D992787FD90950E9436
:10122000F91CB8AEAFAA1A821982AFA8B8AC13C025
:10123000F5E24F1649F481E090E09A8389832AE031
:101240002BAF3324552407C0B301842D992787FD84
:1012500090950E94F91C4DAD5EAD4F5F5F4F5EAF44
:101260004DAFF301838183FF04C0EDADFEAD44902B
:1012700003C0EDADFEAD4080442009F002CCF30187
:101280008681978114C0C22E5524EC2DFF27E7FDDF
:10129000F095EC0FFD1F108AB2CCEC2DFF27E7FD77
:1012A000F095EC0FFD1F108AFEEF4F0E92CCEE96DC
:1012B0000FB6F894DEBF0FBECDBFDF91CF911F9167
:1012C0000F91FF90EF90DF90CF90BF90AF909F90E5
:1012D0008F907F906F905F904F903F902F900895E8
:1012E000CF92DF92EF92FF920F931F93CF93DF93F2
:1012F000EC016B017A018901141615060CF072C01D
:1013000090E020E030E060E070E050E2462F66239D
:1013100049F027703070232B29F4FE01E90FF11DED
:1013200050839F5F9601240F311DDE01A90FB11D6F
:10133000F9018081E82FFF27F295E295EF70EF2702
:10134000FF70EF27E050FF4F80818C939F5FDE019D
:10135000A90FB11DF9018081E82FFF27EF70F07010
:10136000E050FF4F80818C939F5F4F3028F4FE0147
:10137000E90FF11D50839F5F4F5F242F33276F5F6D
:101380007F4F2E153F0514F2E92FFF279F012017ED
:10139000310764F4E92FFF2780E2EC0FFD1F808303
:1013A0009F5FE92FFF27E017F107BCF3EC0FFD1F4C
:1013B00010821016110684F490E0E0E0F0E0EC0FEB
:1013C000FD1F8081803311F0803249F49F5FE92F47
:1013D000FF27E017F1079CF381E090E009C080E06F
:1013E00090E006C090E020E030E0E0E0F0E0CFCF19
:1013F000DF91CF911F910F91FF90EF90DF90CF90F1
:1014000008956F927F928F929F92AF92BF92CF92E8
:10141000DF92EF92FF920F931F93CF93DF937C01A4
:101420004B016A0139011416150614F5BB24E0E0DE
:10143000F0E09EE2A92E87010E0F1F1FE80DF91D97
:101440008081F8018083803269F0C82FDD27C7FDD5
:10145000D095CE010E94AF20892B21F4CE01C097F8
:101460000A97B8F4B394EB2DFF27EC15FD051CF398
:101470004C2DEC2DFF27E615F7059CF480E2EE0DD0
:10148000FF1D80834F5FE42FFF27E615F705BCF3B0
:1014900008C0CE010E94D020892B21F7F801A0823C
:1014A000E1CFEE0DFF1D108280E090E0DF91CF9143
:1014B0001F910F91FF90EF90DF90CF90BF90AF9072
:1014C0009F908F907F906F9008958F929F92AF9290
:1014D000BF92CF92DF92EF92FF920F931F93CF9321
:1014E000DF93EA01452B09F463C07C018B0145E8D9
:1014F000A42E46E0B42E35ECC32E36E0D32E21E1E7
:10150000822E21E0922EC031D10580F120E330E01F
:1015100040E150E0B80185E896E00E94700920E1C2
:1015200030E040E150E0B80185EC96E00E94010A0D
:10153000DF92CF92BF92AF92FF92EF929F928F92E3
:101540000E94261D60978DB79EB708960FB6F89437
:101550009EBF0FBE8DBF209759F180E190E0E80E4D
:10156000F91E005F1F4FC031D10580F620E330E047
:10157000AE01B80185E896E00E94700920E130E0F4
:10158000AE01B80185EC96E00E94010ADF92CF928D
:10159000BF92AF92FF92EF929F928F920E94261D70
:1015A0008DB79EB708960FB6F8949EBF0FBE8DBF3D
:1015B00080E090E0DF91CF911F910F91FF90EF902D
:1015C000DF90CF90BF90AF909F908F900895E5E609
:1015D000F0E08081806180830895E5E6F0E080811D
:1015E0008F7E80830895E5E6F0E08081877F8083A9
:1015F0000895E5E6F0E08081886080830895209179
:10160000E5063091E6062F5F3F4F280F391F809186
:10161000E5069091E60682179307C9F708951F9291
:101620000F920FB60F9211248F939F938091E5062E
:101630009091E60601969093E6068093E5068091E8
:101640000207909103070196909303078093020786
:101650009F918F910F900FBE0F901F90189512BE03
:1016600086B7836086BF87B7826087BF8DE083BF00
:1016700083E781BF12BE0895CF93DF93EC01EC8125
:10168000FD81828184FFB3C0838199278B5F9F4F47
:1016900009F4ADC0DF0114968481813009F4A7C03C
:1016A000823009F4A4C0833009F0A1C0ED01898122
:1016B000882309F49CC0813099F18230F1F18330A4
:1016C00011F1843009F446C0853009F450C08630E9
:1016D00009F45AC0873009F464C0883009F46EC038
:1016E000893009F478C08A3009F081C080E090E147
:1016F000AEE0B0E080939B0590939C05A0939D0580
:10170000B0939E0574C080E895E2A0E0B0E08093BD
:101710009B0590939C05A0939D05B0939E0567C083
:1017200080E699E0A0E0B0E080939B0590939C0553
:10173000A0939D05B0939E055AC080EC92E1A0E075
:10174000B0E080939B0590939C05A0939D05B0937A
:101750009E054DC080E09BE4A0E0B0E080939B0537
:1017600090939C05A0939D05B0939E0540C080E09A
:1017700096E9A0E0B0E080939B0590939C05A09330
:101780009D05B0939E0533C080E091EEA0E0B0E0EF
:1017900080939B0590939C05A0939D05B0939E0517
:1017A00026C080E092ECA1E0B0E080939B0590938E
:1017B0009C05A0939D05B0939E0519C080E094E818
:1017C000A3E0B0E080939B0590939C05A0939D05BA
:1017D000B0939E050CC080E098E0A7E0B0E0809355
:1017E0009B0590939C05A0939D05B0939E05DF916A
:1017F000CF910895EF92FF920F931F937B018C017D
:10180000EE0CFF1C001F111FEE0CFF1C001F111F10
:10181000EE0CFF1C001F111FEE0CFF1C001F111F00
:1018200060E070E081EE90E0A80197010E945420F2
:10183000A801970156954795379527956217730725
:101840008407950748F060E070E081EE90E0A80121
:1018500097010E9454200AC060E070E081EE90E0A1
:10186000A80197010E94542021503040832F9927CE
:1018700080939800209399001F910F91FF90EF9013
:101880000895682F80E00E949C1780E090E0089502
:10189000682F81E00E949C170895CF92DF92FF92FB
:1018A0000F931F93CF93DF93EC010E94F013B3E0EB
:1018B000CB2ED12CCC0EDD1E2B8199279F938F939D
:1018C0003327FE01E20FF31F848199279F938F93A3
:1018D0003F932F938A8199279F938F93898199278B
:1018E0009F938F93888199279F938F9381E291E0B3
:1018F0009F938F930E94261DFA808DB79EB70E96F8
:101900000FB6F8949EBF0FBE8DBFFF2009F46DC0C7
:1019100085E791E09F938F930E94261D0F2D11273D
:101920000F900F9000FD13C001FD1BC002FD23C0EE
:1019300003FD2BC004FD33C005FD3BC006FD43C0C5
:10194000F7FC4AC08AE090E00E94751D4EC08BE80B
:1019500091E09F938F930E94261D0F900F9001FF9F
:10196000E5CF80E991E09F938F930E94261D0F9011
:101970000F9002FFDDCF86E991E09F938F930E9445
:10198000261D0F900F9003FFD5CF8EE991E09F9316
:101990008F930E94261D0F900F9004FFCDCF85EAF4
:1019A00091E09F938F930E94261D0F900F9005FF4B
:1019B000C5CF8EEA91E09F938F930E94261D0F90D2
:1019C0000F9006FFBDCF88EB91E09F938F930E940D
:1019D000261D0F900F90B4CF8FEB91E09F938F93C4
:1019E0000E94261D0F900F90ADCFF6014081552724
:1019F0004B5F5F4FBE0180E090E00E94650ADF917F
:101A0000CF911F910F91FF90DF90CF9008952F926B
:101A10003F924F925F926F927F928F929F92AF927E
:101A2000BF92CF92DF92EF92FF920F931F93CF93CB
:101A3000DF93CDB7DEB72C970FB6F894DEBF0FBE9D
:101A4000CDBF182F8D3079F18A3069F18830A1F03F
:101A500060918E0770918F070E94410C8091040560
:101A6000E82FFF27E75EFA4F10838F5F809304050E
:101A7000803809F03FC5B8C080910405882309F477
:101A800039C580EA90E09F938F930E94461DE091B4
:101A90000405E150E0930405FF27E75EFA4F10824A
:101AA0000F900F9027C560918E0770918F078AE085
:101AB0000E94410CE0910405FF27E75EFA4F108277
:101AC00080911905882309F472C010920505E0E0A1
:101AD000F0E089E195E015E0812E15E0912E94016A
:101AE0007C01DC018C91882309F46CC0803209F4FC
:101AF00069C0D9018D939D013196C7010196E431EA
:101B0000F10571F710921805EE24FF2405E015E0A9
:101B100080910505882309F44AC066EC71E0C8018C
:101B20000E94771C892B09F474C043E050E068ECF4
:101B300071E0C8010E94811C892B09F073C0E11477
:101B4000F104A9F1F701D080F80101900020E9F734
:101B50003197E550F540379708F49AC100E0BB246F
:101B600097012F5F3F4FF7018181803231F42F5F62
:101B70003F4FD9018C918032D1F3A091EF04B09105
:101B8000F004F90101900020E9F73197E21BF30B13
:101B9000CE2E7901FD0123854D2D6B2DCD010E94A7
:101BA000AE1487FD98C183EE91E00E947C1D84EA0B
:101BB00090E09F938F930E94461D109204050F9012
:101BC0000F9098C4EB5FFA4F1082F701808180324A
:101BD00039F40894E11CF11CD7018C918032C9F3CF
:101BE000882309F093CF90CF109204051092190525
:101BF00087E990E09F938F930E94461D84EA90E0CE
:101C00009F938F930E94461D0F900F900F900F90FF
:101C100071C483E091E09F938F930E94461D0F90C3
:101C20000F90C5CF44E050E06FEE71E0C8010E9414
:101C3000811C892B09F05FC1E114F10409F414C37C
:101C4000D701DD903D01F7018181803239F408949C
:101C5000611C711CD3018C918032C9F3F301019096
:101C60000020E9F73197E619EB83F4010190002099
:101C7000E9F73197E550F540359708F0CBC1F4E02E
:101C8000BF2EE090EB04F090EC040091ED04109175
:101C9000EE0417FDCCC1C801B7010E9403209B01CF
:101CA000AC0160E070E080E89FE30E94FE1720E056
:101CB00030E040E451E40E94761F20E030E040E84C
:101CC00052E40E94761F20E030E04AE754E40E948C
:101CD000761F23E333E343E95FE30E94761F20E0AE
:101CE00030E040E85FE30E94BF1F0E94CB1E1B0153
:101CF000B0E0EB16B2ECFB06B1E00B07B0E01B075F
:101D000008F4E4C0E8EEF3E0FC87EB8710920307E9
:101D1000109202071C82442455241E821D821886BC
:101D20001F821A8619862CC08D819E8101969E8302
:101D30008D83E091EF04F091F004848195810E94FD
:101D4000F013E091EF04F091F0040480F581E02DB0
:101D50002381E20FF11D9481891729F0AF81B885A5
:101D60001196B887AF83BC81BB2311F42B5F2C8302
:101D70000894411C511C2B853C8542165306D8F40F
:101D8000E091EF04F091F00481E08F93410121E0B4
:101D9000A22ECB8073010B2D23854D2D60E0CF014A
:101DA0000E9466150F9087FFBFCFE985FA853196AF
:101DB000FA87E987DDCF4090020750900307B20110
:101DC000882777FD8095982F0E9403203B014C01C6
:101DD00057FC44C1AB85BC85BD01882777FD809544
:101DE000982F0E9403205B016C019B01AC01C40190
:101DF000B3010E94FE177B018C0120E030E040E03F
:101E00005FE30E94761F9F938F937F936F931F933F
:101E10000F93FF92EF92A4019301C601B5010E94B6
:101E2000FE1720E030E04AE754E40E94761F9F93BB
:101E30008F937F936F935F924F92E985FA85FF931B
:101E4000EF932F8138853F932F938D819E819F93B0
:101E50008F93AB85BC85BF93AF93BC818B2F9927A4
:101E60009F938F93EB818E2F992705969F938F9346
:101E700084E192E09F938F930E94261D2DB73EB779
:101E8000245E3F4F0FB6F8943EBF0FBE2DBF8FCEDE
:101E9000BB2463E670E0C8010E946B1C892B11F023
:101EA000B1E0BB2E61E670E0C8010E946B1C892B7B
:101EB00009F4D8C104E069E670E085E095E00E948D
:101EC0006B1C892B09F44CCE08604ACE24E630E026
:101ED0003C872B871BCF992787FD90959F938F93E6
:101EE0008CEC91E09F938F930E94261D0F900F9092
:101EF0000F900F905CCE6CEC72E0C8010E94771CD2
:101F0000892B09F0B9C0E114F10409F4B0C0D7017C
:101F1000DC904701F40111810894811C911C812FF0
:101F2000992787FD90950E94C120892B99F711234D
:101F300009F49DC0E091EF04F091F004CC24EE246C
:101F4000FF2408E023854D2D60E0CF010E94AE14F0
:101F5000662477249AE1492E93E0592E3DC08AE108
:101F6000C82E03EFE02E02E0F02E04E02385D4011A
:101F70004C9161E0CF010E94AE14182FE82EFF248F
:101F8000E7FCF094FF92EF927F926F925F924F92F4
:101F90000E94261DEDB7FEB736960FB6F894FEBF29
:101FA0000FBEEDBF111664F4FF92EF9280E393E051
:101FB0009F938F930E94261D0F900F900F900F906C
:101FC0008AE090E00E94751D0894611C711CF4E188
:101FD0006F16710409F4EBCDE091EF04F091F00479
:101FE0008585882309F4BBCF8EE093E00E947C1D99
:101FF000E091EF04F091F004848195810E944D0CF2
:10200000E091EF04F091F0041586E091EF04F09177
:10201000F004A5CF69E670E085E095E004960E94A3
:102020006B1C892B09F42BCEACE0BA2E2ACEC8014A
:10203000B7016170707080709070A801970156951B
:10204000479537952795622B732B842B952B0E94F0
:1020500003209B01AC010E94BF1F21CE20E030E095
:1020600040E857E40E94BF1F3B014C01B3CE84ED12
:1020700092E00E947C1D9BCD67E573E0C8010E9441
:10208000771C892B09F0F5C02091EB043091EC040A
:102090004091ED045091EE0457FD8EC1CA01B90183
:1020A0000E9403209B01AC0160E070E080E89FE3A8
:1020B0000E94FE1720E030E040E151E40E94761FCC
:1020C00020E030E040E852E40E94761F20E030E05B
:1020D0004AE754E40E94761F2DEC3CEC4CE85FE3A9
:1020E0000E94761F20E030E040E85FE30E94BF1FBF
:1020F0000E94CB1E2B017F936F938CE593E09F93FF
:102100008F930E94261DDD24662477240F900F9064
:102110000F900F9034C0892F99279F938F93822F10
:1021200099279F938F93FD01818199279F938F9387
:1021300081E893E09F938F930E94261DE091EF0426
:10214000F091F0040480F581E02D438155274B5F29
:102150005F4FBF0180E090E00E94650A2DB73EB757
:10216000285F3F4F0FB6F8943EBF0FBE2DBF0894B7
:10217000611C711C3FEF6316710409F49FC0E0916C
:10218000EF04F091F004838599278615970579F37C
:102190007F926F9288E793E09F938F930E94261D12
:1021A000E091EF04F091F00481E08F934201B1E0FF
:1021B000AB2ECC24EE24FF240CE02385462D60E0DA
:1021C000CF010E9466150F900F900F900F900F9007
:1021D00087FDCDCFE091EF04F091F00484819581EB
:1021E0000E94F013982FE091EF04F091F004A48185
:1021F000B581FD018381482F5527E40FF51F248108
:10220000921709F088CF06E017E01496BD01C801C7
:102210000E948F1CC3010E94B920892BD1F07F92AC
:102220006F928EEA93E09F938F930E94261D0F90EA
:102230000F900F900F901F930F938FEB93E09F934E
:102240008F930E94261DD3940F900F900F900F90A4
:102250008ECF87EB93E09F938F930E94261D0F9064
:102260000F90E9CF00E027CE84EF91E00E947C1D23
:102270009ECC6DED73E0C8010E94771C892BB9F5E7
:10228000E114F10409F4ADC0E091EF04F091F00421
:10229000D7018C918387E091EF04F091F00483855E
:1022A00099279F938F938EEF93E09F938F930E9434
:1022B000261D0F900F900F900F9079CC85EC93E036
:1022C0009F938F930E94261D8D2D99279F938F9307
:1022D0008DEC93E09F938F930E94261D8DB79EB740
:1022E00006960FB6F8949EBF0FBE8DBF60CC60E21D
:1022F00074E0C8010E94771C892BF1F5E114F10408
:1023000001F140E050E0BE016F5F7F4FC7010E94C6
:102310000D1B9B01AC01E981FA81EE16FF0621F04D
:102320008081882309F470C0FF92EF9280E494E0EA
:102330009F938F930E94261D0F900F900F900F90E8
:1023400036CC8091EB049091EC04A091ED04B09117
:10235000EE04BF93AF939F938F9385E294E09F9396
:102360008F930E94261DEDB7FEB736960FB6F894F0
:10237000FEBF0FBEEDBF1BCC6AE974E0C8010E942E
:10238000771C892B81F48091EA0490E0882309F47A
:1023900091E09093EA04992309F49CC08CE994E0BD
:1023A0000E947C1D04CC80E990E09F938F930E9453
:1023B000461D0F900F90FBCBCA01B9016170707080
:1023C000807090705695479537952795622B732BA3
:1023D000842B952B0E9403209B01AC010E94BF1F00
:1023E00061CEE091EF04F091F004838599279F93EB
:1023F0008F9380EE93E09F938F930E94261D0F9002
:102400000F900F900F90D3CB2093EB043093EC04FC
:102410004093ED045093EE04CA01B9010E94FA0BF7
:102420008091EB049091EC04A091ED04B091EE0446
:10243000BF93AF939F938F9380E694E09F938F9386
:102440000E94261DE090EB04F090EC040091ED0456
:102450001091EE04EE0CFF1C001F111FEE0CFF1C70
:10246000001F111FEE0CFF1C001F111FEE0CFF1CA4
:10247000001F111F60E070E081EE90E0A80197015D
:102480000E945420A80197015695479537952795A6
:10249000ADB7BEB716960FB6F894BEBF0FBEADBFB0
:1024A0006217730784079507D0F060E070E081EE53
:1024B00090E0A80197010E9454203F932F938CE74E
:1024C00094E09F938F930E94261D0F900F900F9082
:1024D0000F906DCB81EB94E00E947C1D68CB60E097
:1024E00070E081EE90E0A80197010E9454202150F5
:1024F0003040E3CF2C960FB6F894DEBF0FBECDBFB1
:10250000DF91CF911F910F91FF90EF90DF90CF90CF
:10251000BF90AF909F908F907F906F905F904F9003
:102520003F902F900895CFEFD0E1DEBFCDBF0E9446
:102530002F0BB89AC09A80916400886180936400E0
:10254000809165008F7E8093650080916500877F14
:10255000809365001092E7068091EF049091F0045B
:1025600090939A05809399050E94D913E091EF0406
:10257000F091F00487EE9AE0918B808B8DEE9AE0DB
:10258000938B828B83EF9AE0958B848B89EF9AE013
:10259000978B868B88E49CE0918F808FE090EB0492
:1025A000F090EC040091ED041091EE04EE0CFF1C91
:1025B000001F111FEE0CFF1C001F111FEE0CFF1C53
:1025C000001F111FEE0CFF1C001F111F60E070E0C8
:1025D00081EE90E0A80197010E945420A801970184
:1025E0005695479537952795621773078407950782
:1025F00008F4D3C060E070E081EE90E0A80197019C
:102600000E945420B9018FE590E00E94D917789478
:1026100060E070E081E49CE00E94A91CC0988DED10
:1026200090E09F938F930E94461D84EA90E09F93D1
:102630008F930E94461D0F900F900F900F90E09186
:10264000EF04F091F004C6E0D7E007ECA02E04E020
:10265000B02E8585882321F4809181078823C9F3D2
:1026600085858823B9F480918107882371F0F894D7
:10267000109281077894C09802C00E94070D82E8EA
:1026800097E00E94BE168823C1F7E091EF04F09115
:10269000F004DFCFF8940480F581E02D43815527C5
:1026A0004B5F5F4FBF0181E497E00E94621CE091A5
:1026B000EF04F091F00486851586789481E497E024
:1026C0000E94F01310914407412F5527FA01EF5B48
:1026D000F84F24819091430792FD23C020E030E021
:1026E00010E000E080E093FD2DC0882381F0000021
:1026F000E091EF04F091F004C12E7901238540911F
:10270000420760E0CF010E94AE1487FD2FC0809188
:10271000EA04882309F4A7CF81E497E00E944D0CD6
:10272000A2CF821709F102E065E477E086E097E046
:102730000E94621C26E037E0E90181E090914307A6
:1027400093FFD3CF6CEA70E086E097E00E943A1CDA
:10275000FE0101900020E9F73197E650F7401E2F67
:1027600026E037E0E901C3CF01E0DECF992787FDFE
:1027700090959F938F938091420799279F938F9372
:10278000BF92AF920E94261D8DB79EB706960FB6D8
:10279000F8949EBF0FBE8DBFBACF60E070E081EEAF
:1027A00090E0A80197010E945420B9016150704047
:1027B0002ACFFC011682178210861386148615868E
:1027C0001686178681EE95E09183808381EA95E0F5
:1027D0009583848381E296E09383828311860895B2
:1027E000DC01FC0133813C5F9C91323048F021E0F8
:1027F000FD01E20FF11D8081980F2F5F3217C1F7A5
:10280000892F992708951F920F920FB60F921124C6
:102810008F939F93AF93BF93CF93DF93EF93FF93E8
:10282000A0919905B0919A05109791F0ED019F81C3
:102830008885981799F0FD0187810280F381E02D4A
:10284000E80FF11D908190939C008F5FED018F83C5
:1028500080919B00806480939B0002C081E08C8704
:10286000FF91EF91DF91CF91BF91AF919F918F91A8
:102870000F900FBE0F901F9018951F93CF93DF936B
:10288000EC01162FE889F98909950000112389F0D8
:1028900081E08F871C8681E08F83C09AEA81FB816B
:1028A000288D398D8081F90109958C858823E9F37C
:1028B00005C01F86EE89FF890995ECCFC098EA898B
:1028C000FB890995EC89FD890995DF91CF911F91CD
:1028D0000895FC011092E6061092E5066F5F7F4FA7
:1028E0008585882339F48091E5069091E606861760
:1028F0009707B0F38585882319F080E090E008956C
:102900008FEF9FEF0895CF93DF93EC010E9469143E
:10291000882319F08FEF9FEF0AC0EC81FD8182813F
:1029200080FF03C080E090E002C08EEF9FEFDF9158
:10293000CF910895EF92FF920F931F937C018B012B
:102940000E94FD1A0E191F09B8010E942D208E0D3C
:102950009F1D1F910F91FF90EF900895CF92DF92EE
:10296000EF92FF920F931F93CF93DF93EC01D62E3C
:102970003C2D8C2D9927CC970CF097C0EA81FB81D8
:102980008AEA8083EA81FB818183EA81FB818283F9
:10299000EA81FB8189E98383EA81FB814483EA81BF
:1029A000FB812583240FEA81FB810683200FEA81C6
:1029B000FB81C7822C0DCC2009F043C0E8E0F0E099
:1029C00039E08A819B81E80FF91F20833887DD2059
:1029D00009F453C0EE24FF240E2D1D866D2DCE016B
:1029E0000E943D141F861092E6061092E5068D8522
:1029F000813031F08091E5069091E6060597B8F3B5
:102A00008D85882309F040C091E0C92E68E270E00E
:102A10008AE090E00E949A148C018AE290E00E9481
:102A2000751DC8010E94FF0A0894E11CF11C86E094
:102A3000E816F10489F6C1948C2D992787FD9095AD
:102A40003CC0D7019C2D8A2F8E19885FEA81FB81BB
:102A5000E80FF11D8C9180838D91280F915099F78B
:102A6000385FE32FFF273F5F8A819B81E80FF91FC3
:102A700020833887DD2009F0ADCF60E0CE010E94D1
:102A80003D1480E090E019C0EA81FB8134964381D7
:102A900055274B5F5F4FBF018C819D810E94551C64
:102AA000892B31F082E0C82EB1CF8FEF9FEF05C0A8
:102AB0001D86802F992787FD9095DF91CF911F91DB
:102AC0000F91FF90EF90DF90CF9008952F923F925B
:102AD0004F925F926F927F928F929F92AF92BF922E
:102AE000CF92DF92EF92FF920F931F93CF93DF93DA
:102AF000CDB7DEB721970FB6F894DEBF0FBECDBFBE
:102B00003C016983242E322EB02E2701DC2CAA2012
:102B1000C1F010E009C0B401C3010E9483148823EE
:102B200099F01F5FA11669F0F3011586CD2C720193
:102B30000B2D232D422D6981C3010E94AE1487FF06
:102B4000EACF8FEF9FEF07C08E89882311F0F30142
:102B5000158680E090E021960FB6F894DEBF0FBE98
:102B6000CDBFDF91CF911F910F91FF90EF90DF903C
:102B7000CF90BF90AF909F908F907F906F905F901D
:102B80004F903F902F9008951F920F920FB60F9283
:102B900011241F932F933F934F935F936F937F93D2
:102BA0008F939F93AF93BF93CF93DF93EF93FF9355
:102BB00010919B0020919C00C0919905D0919A059D
:102BC000209791F08985833029F1843090F0853009
:102BD00009F466C08530A0F1863009F478C08730EA
:102BE00009F48EC0C098198616FFB4C00E94031461
:102BF000B1C0813009F44DC0823068F1C09A209391
:102C0000A0058B852817C1F18F858823A9F583E05E
:102C10008987EACF9B858091A005981719F08F8549
:102C2000882359F08E81E881F981E80FF11D208316
:102C30008F5F8E838A85280F2A8784E08987D4CF87
:102C40009B858091A005981759F08F85882341F4C2
:102C500085E08987C9CF2A3A39F681E08987C4CFD0
:102C60008E81E881F981E80FF11D20838F5F8E83CB
:102C70008A85280F2A87ECCF1E821E861D868E81AC
:102C8000E881F981E80FF11D20838F5F8E832A8709
:102C9000BECF293991F12A3A09F4A6CF1986A4CFDB
:102CA0008E81E881F981E80FF11D20838F5F8E838B
:102CB0008A85820F8A8720939F052223D9F0822F4D
:102CC0009927CD970CF08FCF86E089878DCF8E81A5
:102CD000E881F981E80FF11D20838F5F8E838A855B
:102CE000280F2A8780919F05815080939F05882314
:102CF00009F07ACF87E0898777CF82E0898774CF20
:102D00008E81E881F981E80FF11D20839B858091F8
:102D1000A005981719F08F858823C9F09A858E81B0
:102D2000A881B981FD01E80FF11D8081981711F08C
:102D300081E08E87FD01438155274B5F5F4FBD01C9
:102D40008C819D810E94621C81E08D871986C098CC
:102D500019864ACFFF91EF91DF91CF91BF91AF914B
:102D60009F918F917F916F915F914F913F912F91A3
:102D70001F910F900FBE0F901F901895CF93DF9368
:102D8000DC01EC018A819B81892BF1F0ED01EE8160
:102D9000FF816191FF83EE838A819B8101979B83F1
:102DA0008A834E815F81888599852D913C91820F20
:102DB000931F4817590718F4862F992707C088854D
:102DC00099859F838E83F8CF80E090E0DF91CF914B
:102DD0000895FC01518340831382128275836483BA
:102DE00077836683718760870895FC018281938170
:102DF000892B31F00680F781E02D80819927089595
:102E000080E090E00895CF93DF93DC01EC012A810C
:102E10003B818D919C91119728173907C8F4EC815B
:102E2000FD816193FD83EC838A819B8101969B8365
:102E30008A834C815D81888599852D913C91820F93
:102E4000931F4817590720F0888599859D838C83A7
:102E5000DF91CF910895CF93DF93DC01EC018A815C
:102E60009B81892BF1F0ED01EE81FF8161917191E0
:102E7000FF83EE838A819B8101979B838A834E81A6
:102E80005F81288539858D919C91880F991F280F26
:102E9000391F4217530738F0888599859F838E83A1
:102EA00002C060E070E0CB01DF91CF910895FC019A
:102EB0005183408313821282758364837783668390
:102EC000718760870895FC0182819381892B31F09D
:102ED0000680F781E02D80819181089580E090E067
:102EE0000895CF93DF93DC01EC012A813B818D9122
:102EF0009C91119728173907E0F4EC81FD816193CB
:102F00007193FD83EC838A819B8101969B838A83E5
:102F10004C815D81288539858D919C91880F991F01
:102F2000280F391F4217530720F0888599859D8304
:102F30008C83DF91CF910895882319F0813029F097
:102F400008955D9BFECF6CB9089580919B0085FF2D
:102F5000FCCF60939C0008951F920F920FB60F92C2
:102F600011242F933F934F935F936F937F938F938E
:102F70009F93AF93BF93EF93FF93C09A6CB15C990B
:102F800007C082E897E00E94031781E080938107E1
:102F9000FF91EF91BF91AF919F918F917F916F9131
:102FA0005F914F913F912F910F900FBE0F901F9007
:102FB0001895EF92FF920F931F938C017B0140E2D3
:102FC00050E065E676E082E897E00E94E91610920C
:102FD0008107812F99278093900009B988E98AB9E0
:102FE0008F2D992780939800E092990088ED809327
:102FF0009A001F910F91FF90EF900895A8E1B0E023
:10300000E4E0F8E10C947C2069837A838B839C83D1
:103010002D833E834F835887B9E08B2E912C8C0EE5
:103020009D1EB401CE0101960E940A1A8E010F5E08
:103030001F4FB801CE0105960E940A1A2985223039
:1030400008F46AC03989323008F468C08A859A89E0
:1030500089278A87243009F463C0223009F460C0CC
:10306000343041F41D861E861F86188A1C861B86F6
:10307000B40177C0323009F458C06B857C858B89E8
:103080009C89681B790B7C876B872D853E854F85D6
:103090005889ED88FE880F89188D2E153F05400749
:1030A000510740F4220F331F441F551F61507040D9
:1030B0007C876B8780E090E0A0E0B0E4AA24BB248A
:1030C000650160E070E02E153F054007510740F0B4
:1030D000A82AB92ACA2ADB2A2E193F09400B510B0C
:1030E000B695A79597958795220F331F441F551FB7
:1030F0006F5F7F4F6F31710531F7D601C5018F7753
:103100009070A070B07080349105A105B10589F070
:10311000AD86BE86CF86D88AB40123C0B80121C04F
:103120003217D1F761EF74E01CC084E08987B401E5
:1031300018C0A7FCEDCF211531054105510541F31C
:1031400080E490E0A0E0B0E0A80EB91ECA1EDB1E2D
:1031500080E89FEFAFEFBFEFA822B922CA22DB229F
:10316000D7CFCB010E94E818ECE068960C94982029
:10317000A8E1B0E0EEEBF8E10C94862069837A8355
:103180008B839C832D833E834F835887BE01675F6B
:103190007F4FCE0101960E940A1ABE016F5E7F4FDB
:1031A000CE0105960E940A1A8985823018F481E0C2
:1031B00090E00AC020E030E08989823010F0C90137
:1031C00003C021E030E0C901E2E068960C94A2203F
:1031D0004F925F926F927F928F929F92AF92BF9227
:1031E000DF92EF92FF920F931F9320E030E040E0D8
:1031F00050E0FC01E480F58006811781D180808158
:10320000823038F4D801C701A061AF77B0706FEF9A
:10321000D9C0843009F46EC0823009F471C0E11461
:10322000F1040105110509F46BC0828193816FEFF0
:10323000823896070CF06AC062E87FEF681B790B52
:103240006A3171050CF080C047015801062E04C098
:10325000B694A794979487940A94D2F7442455245B
:10326000320181E090E0A0E0B0E004C0880F991F37
:10327000AA1FBB1F6A95D2F70197A109B109E822DD
:10328000F9220A231B23E114F1040105110529F099
:1032900061E0462E512C612C712C85017401E428CB
:1032A000F52806291729D801C7018F779070A070DB
:1032B000B07080349105A105B10509F457C0D8015B
:1032C000C701CF96A11DB11D60E070E08030E0E045
:1032D0009E07E0E0AE07E0E4BE0710F061E070E0BA
:1032E00027E0B695A795979587952A95D1F7AF775B
:1032F000B07068C080E090E0A0E0B0E06FEF62C026
:1033000080E090E0A0E0B0E060E05CC08038910533
:103310008CF7BC0161587F4FD801C7018F7790703F
:10332000A070B07080349105A105B105A1F08FE3C4
:1033300090E0A0E0B0E0E80EF91E0A1F1B1F17FD89
:1033400028C0D801C701CCCF60E070E080E090E0F9
:10335000A0E0B0E0CCCFE7FEF2CF80E490E0A0E0C8
:10336000B0E0E80EF91E0A1F1B1FE9CFE7FC18C0EA
:1033700080E090E060E0E61660E0F60660E00607B8
:1033800060E4160710F081E090E0BC01D801C701AD
:10339000A7CF16950795F794E7946F5F7F4FD1CF2E
:1033A000D801C701805C9F4FAF4FBF4F60E070E016
:1033B0008030E0E09E07E0E0AE07E0E4BE0708F4FE
:1033C0008FCF8CCF282F392F9A2F9F77842F8078FB
:1033D000892B962F9795992797958F77482F492B6B
:1033E0006695852F8078862BD794DD24D7948F77A8
:1033F000582F5D29CA01B9011F910F91FF90EF90DD
:10340000DF90BF90AF909F908F907F906F905F9074
:103410004F900895FC01DB01208131819281492F79
:103420004F7750E0991F9927991F8381682F660F66
:10343000692B881F8827881FFD018183662309F077
:1034400049C0211531054105510509F470C082E8D4
:103450009FEFFD0193838283220F331F441F551F6B
:10346000220F331F441F551F220F331F441F551FA8
:10347000220F331F441F551F220F331F441F551F98
:10348000220F331F441F551F220F331F441F551F88
:1034900083E08C932030F0E03F07F0E04F07F0E44A
:1034A0005F0790F482E89FEF220F331F441F551FE0
:1034B0000197203060E0360760E0460760E4560779
:1034C00098F3FD0193838283FD0124833583468332
:1034D000578308956F3F71F1862F99278F5790403A
:1034E000FD019383828383E08C93220F331F441F5B
:1034F000551F220F331F441F551F220F331F441F18
:10350000551F220F331F441F551F220F331F441F07
:10351000551F220F331F441F551F220F331F441FF7
:10352000551F50642483358346835783089582E072
:103530008C930895211531054105510519F484E056
:103540008C93089544FD02C01C92BECF81E08C9301
:10355000BBCFAF92BF92CF92DF92EF92FF920F93C9
:103560001F93CF93DF93EC01E880F9800A811B81E0
:10357000C801B7012DE133EF41E050E00E94542033
:1035800027EA31E440E050E00E94EE205B016C014C
:10359000C801B7012DE133EF41E050E00E94542013
:1035A000CA01B90124E13BE040E050E00E94EE2076
:1035B000A61AB70AC80AD90A1A141B041C041D0447
:1035C00044F08FEF9FEFAFEFBFE7A80EB91ECA1E02
:1035D000DB1EA882B982CA82DB82C5019F77DF9198
:1035E000CF911F910F91FF90EF90DF90CF90BF9000
:1035F000AF9008950E94A91A089589EF94E00E945F
:10360000A91A0895AA27BB278093F9049093FA0476
:10361000A093FB04B093FC0408953F924F925F92F5
:103620006F927F928F929F92AF92BF92CF92DF92D2
:10363000EF92FF920F931F93CF93DF938C012B0197
:10364000EA016115710519F0FB01918380832097D0
:1036500049F0CE010297839728F060E070E080E0A7
:1036600090E0F6C0F801E1908F018E2D99270E941D
:10367000C120892BB9F7FDE2EF1631F4F801E19092
:103680008F0181E0382E07C0FBE2EF1619F4F80134
:10369000E1908F013324209719F0C031D105C1F496
:1036A000F0E3EF1679F4F8018081883711F088355E
:1036B00049F4F801E1800E5F1F4FF2E03F2AC0E1BC
:1036C000D0E006C0209721F480E3E816E9F427C093
:1036D000C830D10531F1C930D10524F4C230D1054B
:1036E00031F50CC0CA30D10589F0C031D105F9F4EB
:1036F000A12CB12CC12CB8E0DB2E26C0A12CB12C02
:10370000C12CA0E4DA2E20C0CAE0D0E0FCECAF2E41
:10371000FCECBF2EFCECCF2EFCE0DF2E15C0C8E089
:10372000D0E0A12CB12CC12CE0E1DE2E0DC09E0119
:10373000442737FD4095542F60E070E080E090E82A
:103740000E94542059016A0120E030E040E050E03E
:1037500060E03E01882477FC8094982C70EDF72E71
:10376000FE0CE9E0EF1570F48E2D81548A3118F4C7
:1037700099ECF92E06C08E2D81568A3150F589EAD2
:10378000F82EFE0C8F2D99278C179D0714F567FDD9
:103790001CC0A216B306C406D506B0F0CA01B90112
:1037A000A40193010E94EE209B01AC012F0D311D5D
:1037B000411D511D2130F0E03F07F0E04F07F0E8D8
:1037C0005F0710F461E001C06FEFF801E1908F0135
:1037D000C5CF4114510481F0662331F001501040EF
:1037E000F2011183008308C031FE1AC0025010405C
:1037F000F2011183008314C067FF12C030FE05C0C0
:1038000020E030E040E050E804C02FEF3FEF4FEF02
:103810005FE782E290E0909393078093920716C04F
:1038200030FE08C050954095309521953F4F4F4F41
:103830005F4F0CC057FF0AC082E290E0909393075D
:10384000809392072FEF3FEF4FEF5FE7CA01B90177
:10385000DF91CF911F910F91FF90EF90DF90CF906C
:10386000BF90AF909F908F907F906F905F904F90A0
:103870003F900895FB01DC0105900D920020E1F7D7
:103880000895FC0105900020E9F7809590958E0F32
:103890009F1F0895FC010590615070400110D8F7FA
:1038A000809590958E0F9F1F0895FB01DC0104C049
:1038B0008D910190801921F441505040C8F7881B28
:1038C000990B0895FB01DC0102C001900D9241505B
:1038D0005040D8F70895FC010190061629F0002009
:1038E000D9F78827992708953197CF010895FB01CB
:1038F000DC018D910190801911F40020D1F7990B12
:103900000895FB01DC014150504030F08D91019051
:10391000801919F40020B9F7881B990B0895FB0151
:10392000DC014150504048F001900D920020C9F751
:1039300001C01D9241505040E0F70895FC016150D4
:10394000704001900110D8F7809590958E0F9F1FC1
:103950000895EF92FF920F931F93CF93DF938C0103
:103960007B01892B11F4672BD1F16EE070E081E0CF
:1039700090E00E94AF1DFC01009789F1DC0180E816
:103980008383E114F10471F0F386E28681E8838396
:1039900080918C0790918D07892B21F4F0938D07EE
:1039A000E0938C0701151105E1F0118700878381F1
:1039B0008260838380918E0790918F07892B89F491
:1039C000F0938F07E0938E07809190079091910775
:1039D000892B39F4F0939107E093900702C0A0E09F
:1039E000B0E0CD01DF91CF911F910F91FF90EF904B
:1039F00008950F931F93CF93DF938C01EB018B817D
:103A0000992781FF1BC082FF0DC02E813F818C81D1
:103A10009D812817390764F4E881F9810193F983BE
:103A2000E88306C0E885F985802F0995892B31F454
:103A30008E819F8101969F838E8302C00FEF1FEFBF
:103A4000C801DF91CF911F910F910895CF93DF931C
:103A5000CDB7DEB722970FB6F894DEBF0FBECDBF4D
:103A6000FE01379661917191FA83E983AF018091EC
:103A70008E0790918F070E94150522960FB6F89435
:103A8000DEBF0FBECDBFDF91CF910895CF93DF93FF
:103A9000CDB7DEB722970FB6F894DEBF0FBECDBF0D
:103AA000FE01379661917191FA83E983E0918E0767
:103AB000F0918F0783818860838349815A81809147
:103AC0008E0790918F070E941505E0918E07F09167
:103AD0008F072381277F238322960FB6F894DEBFBA
:103AE0000FBECDBFDF91CF91089560918E07709189
:103AF0008F070E94F91C08950F931F93CF93DF93B4
:103B00008C01E0918E07F0918F07838181FF1FC0A8
:103B1000C0E0D0E00AC0FD0120853185BD01F9017A
:103B20000995892B11F0CFEFDFEFF80181918F011B
:103B3000A0918E07B0918F07882369F7FD0120853A
:103B40003185BD018AE0F9010995892B11F0CFEF8C
:103B5000DFEFCE01DF91CF911F910F9108950F9369
:103B60001F93CF93DF93869F8001879F100D969FB1
:103B7000100D1124C8010E94CB1DEC01009729F003
:103B8000A80160E070E00E94C41ECE01DF91CF91D9
:103B90001F910F910895CF93DF93AC01029710F41A
:103BA00042E050E0A0919607B0919707FD01C0E078
:103BB000D0E020E030E020C080819181841795071B
:103BC00069F482819381209719F09B838A8304C0D2
:103BD0009093970780939607CF0132C048175907F3
:103BE00038F42115310519F08217930708F49C0168
:103BF000EF010280F381E02D3097F1F621153105B8
:103C000089F1C901841B950B049708F4A901E0E030
:103C1000F0E026C08D919C91119782179307E9F4EB
:103C20004817590779F4ED018A819B81309719F083
:103C30009383828304C09093970780939607CD0166
:103C4000029649C0841B950BFD01E80FF91F4193B3
:103C5000519302978D939C933AC0FD01A281B38149
:103C60001097C1F68091940790919507892B41F4A4
:103C70008091FF049091000590939507809394079D
:103C800020910105309102052115310541F42DB730
:103C90003EB78091FD049091FE04281B390BE09102
:103CA0009407F09195072E1B3F0B2417350788F0DA
:103CB000CA0102962817390760F0CF01840F951FBB
:103CC0000296909395078093940741935193CF0167
:103CD00002C080E090E0DF91CF910895CF93DF9311
:103CE000009709F44EC0EC0122971B821A82A09122
:103CF0009607B0919707109711F140E050E001C08E
:103D0000DC01AC17BD0700F1BB83AA83FE01219142
:103D10003191E20FF31FEA17FB0771F42E5F3F4F5B
:103D20008D919C911197820F931F99838883FD0138
:103D3000828193819B838A834115510559F4D093E5
:103D40009707C09396071DC0FD0182819381AD0145
:103D50000097B1F6FA01D383C28321913191E20F2A
:103D6000F31FEC17FD0769F42E5F3F4F888199819F
:103D7000820F931FFA01918380838A819B819383B1
:103D80008283DF91CF910895DC0101C06D93415092
:103D90005040E0F7089597FB47D09F3738F0FEE991
:103DA000F91B982F872F762F6B2F05C05AC0969539
:103DB000879577956795F150D0F73EF4909580956B
:103DC000709561957F4F8F4F9F4F08950ED05EF095
:103DD00004C00BD026F001C008D019F020F48FEFFA
:103DE000089580E0089581E0089597FB092E052647
:103DF00000F8689410D0E89407FC07C062177307B6
:103E00008407950721F008F4009407949894089586
:103E1000052E092607FA440F551F5F3F79F0AA27A0
:103E2000A51708F051E04795880F991F9F3F31F083
:103E3000BB27B91708F091E0879508959F919F914E
:103E4000112408C197FB880F991F9F3F31F0BB27B2
:103E5000B91708F091E0879508959F919F911124DB
:103E6000F9C0662777278827992708959F3F59F437
:103E7000803C49F481E0992708959068892387233D
:103E800086238395B9F3882799270895DBDFCF939D
:103E9000DF93D52FC42F5527442733272227992373
:103EA000D9F09F37C8F0F92FBDD0592F482F372FA1
:103EB000262FF63968F46FDFA6D0C030CD0721F089
:103EC00069937993899399939058DF91CF9157C0D3
:103ED0009927882777276627C030CD0721F02993B7
:103EE000399349935993DF91CF919CC091DF01D0D1
:103EF00099C0992339F0552329F09F575F57950FA3
:103F000013F49AF1B1CF91589F3FE1F3629FA12D35
:103F10000F92BB27639FA00DB11DEE27729FA00DCE
:103F2000B11DEE1FAF93AA27649FB00DE11D739FD3
:103F3000B00DE11DAA1F6627829FB00DE11DA61FCF
:103F40005527749FE00DA11D551F839FE00DA11DF6
:103F5000561F849FA00D511D852F7A2F6E2F1F9005
:103F60000F9088231AF4939539F474C0000C111C37
:103F7000BB1F661F771F881F012808955058192EF0
:103F800047DF01D04FC0BA17620773078407950750
:103F9000B1F188F40EF410940B2EBA2FA02D062E3A
:103FA000622F202D072E732F302D082E842F402DA9
:103FB000092E952F502DFF275523B9F0591B49F095
:103FC000573E98F0469537952795A795F04053951D
:103FD000C9F776F0BA0F621F731F841F30F48795FC
:103FE00077956795B795F040939517FA0F2E08953A
:103FF000BF1BBB27BA0B620B730B840BF6CFDEF62D
:1040000033CFE89403C097FB0EF4D8DEB62F672FAA
:10401000782F892F9EE9002405C09A95BB0F661F53
:10402000771F881F11249923A1F08823B2F79F3F9F
:1040300059F0BB0F48F421F4002011F460FF04C0D4
:104040006F5F7F4F8F4F9F4F881F9795879597F989
:10405000089507CF9FEF80EC0895AA1BBB1B51E189
:1040600007C0AA1FBB1FA617B70710F0A61BB70BE8
:10407000881F991F5A95A9F780959095BC01CD018D
:10408000089597FB092E07260AD077FD04D0E5DFB7
:1040900006D000201AF4709561957F4F0895F6F7C9
:1040A000909581959F4F0895A1E21A2EAA1BBB1BE4
:1040B000FD010DC0AA1FBB1FEE1FFF1FA217B307F4
:1040C000E407F50720F0A21BB30BE40BF50B661F0A
:1040D000771F881F991F1A9469F7609570958095CE
:1040E00090959B01AC01BD01CF0108952F923F92A5
:1040F0004F925F926F927F928F929F92AF92BF92F8
:10410000CF92DF92EF92FF920F931F93CF93DF93A3
:10411000CDB7DEB7CA1BDB0B0FB6F894DEBF0FBE00
:10412000CDBF09942A88398848885F846E847D844D
:104130008C849B84AA84B984C884DF80EE80FD804F
:104140000C811B81AA81B981CE0FD11D0FB6F894C5
:10415000DEBF0FBECDBFED01089585FD36C0806284
:10416000911133C08136ECF38B37DCF70895803240
:1041700039F0992329F480321CF08F370CF408951C
:1041800024C0911122C0803251F08A3041F08C302D
:1041900031F08D3021F0893011F08B3099F708958E
:1041A000082EE7DF41F0EDDF81110FC0802D04D034
:1041B0008823D9F78FEF0895911107C08F9308D006
:1041C00088238F9109F00895CACF992788270895E9
:1041D0009111FBCF80538A50E0F70895629FD00180
:1041E000739FF001829FE00DF11D649FE00DF11DB2
:1041F000929FF00D839FF00D749FF00D659FF00D61
:104200009927729FB00DE11DF91F639FB00DE11D4D
:0A421000F91FBD01CF01112408952C
:10421A003031323334353637383961626364656632
:10422A0000253034782020257320207C25737C0AD1
:10423A00000A494E434F4D494E4720504B543A20AD
:10424A00544F3D3078253032782046524D3D3078F3
:10425A002530327820464C3D30782530327820445B
:10426A00415441204C454E3D256420434B53554D06
:10427A003A20723D307825303278206C3D307825EE
:10428A003032780A002020202020202020202020E0
:10429A00202020464C414753203D002041434B00FB
:1042AA00204E41434B002052455141434B0020527E
:1042BA00455149440020434F4D4D414E4400205240
:1042CA004553455256454400205553455231002026
:1042DA005553455232003F00706B7400706B742066
:1042EA0073656E64206572726F722C2072633D254D
:1042FA00640A00706B742073656E74204F4B0070F3
:10430A00696E670055736167653A2070696E675B0D
:10431A0063695D203C6E6F64653E205B3C6461743A
:10432A00613E5D000A7061636B65742073656E643B
:10433A002073697A65203D2025642062797465734B
:10434A002C207061636B65742072656376207369D3
:10435A007A65203D2025642062797465730A256494
:10436A00207061636B6574732073656E742C2025ED
:10437A00642072656376642C2025642065727273EA
:10438A002C2025642074696D656F7574732C2074F4
:10439A006F74616C206F66202575206D730A25661F
:1043AA00207472616E73616374696F6E73202F205B
:1043BA007365636F6E640A2566206D7320666F727B
:1043CA0020726F756E6420747269700A2566206D9A
:1043DA0073206F6E65207761790A0A00636F6C6CCF
:1043EA006964650075736167653A20636F6C6C690F
:1043FA006465203C6E6F6465313E203C6E6F646577
:10440A00323E0054455354205041434B45542043B7
:10441A004F4C4C4953494F4E204441544100676F19
:10442A0074207061636B65743A002532643A2070B7
:10443A006B745F73656E6428292072633D2564007E
:10444A002C20256420636F6C6C6973696F6E73200E
:10445A00646574656374656420616E642072656363
:10446A006F7665726564007363616E007363616E73
:10447A006E696E67206E6F6465732C2074696D6552
:10448A006F75743D25640A000D3078253032782026
:10449A00000A2162616420636865636B73756D202D
:1044AA0066726F6D206E6F64652025632C203078EC
:1044BA0025327820213D2030782532780A002028BC
:1044CA002725632729200020282E2E2E2920002286
:1044DA002573220A000D20202020200D002575209A
:1044EA006E6F64657320666F756E640A0069640096
:1044FA005253343835206E6F646520616464726586
:10450A007373206973203078253032780A00525349
:10451A00343835206E6F6465206164647265737324
:10452A002073657420746F203078253032780A0041
:10453A00626175640063757272656E74206261757A
:10454A006420726174652069733A20256C640A00DC
:10455A0063616E27742072656164206261756420EC
:10456A00726174652066726F6D20272573270A00B1
:10457A005253343835206261756420726174652043
:10458A0073657420746F20256C640A006261756417
:10459A00207261746520726567697374657220732D
:1045AA00657420746F2025750A007600766572623C
:1045BA006F7365206D6F646520656E61626C6564FA
:1045CA0000766572626F7365206D6F646520646939
:1045DA007361626C656400726573706F6E736520D7
:1045EA00746F206E6F6465202563206661696C654F
:1045FA00642C2072633D25640A000100C20100E8B0
:10460A0006000000000000000001000000200098E1
:04461A000700000095
:00000001FF
